:020000020000FC
:100000001FC218951895189518953DC00CC01895E5
:100010001895189518951895189518951895189578
:100020001895189518950F939F93AF93BF931F93AF
:100030001FB70091630090916000A0916100B091A2
:100040006200003051F49398949895980913939A0C
:100050000A13949A0B13959A09C0091709F49398F7
:100060000A1709F494980B1709F4959803950F3F14
:1000700008F00027009363001FBF1F91BF91AF914D
:100080009F910F9118950F93BF93AF93DF93CF93E9
:100090001F931FB757FD2AC0C29856FF0AC0009190
:1000A000640009BD0091650008BD0FB500620FBD79
:1000B00008C000E009BD00E008BD0FB50F7D0FBD11
:1000C000C49855FF0AC0009166000BBD00916700FF
:1000D0000ABD0FB500680FBD08C000E00BBD00E011
:1000E0000ABD0FB50F770FBDC3984DC0C29A0091DE
:1000F00068000A9509F045C0A8B5B9B556FD05C018
:10010000B03019F4A03009F417C00FB500620FBD6C
:1001100056FF0CC01196D0916400C09165002196E5
:10012000AC17BD0748F02197DE0106C0119721F4F6
:100130000FB50F7D0FBDC498B9BDA8BDAAB5BBB59D
:1001400055FD05C0B03019F4A03009F417C00FB543
:1001500000680FBD55FF0CC01196D0916600C0918C
:1001600067002196AC17BD0748F02197DE0106C055
:10017000119721F40FB50F770FBDC398BBBDAABD72
:1001800008E0009368001FBF1F91CF91DF91AF91EE
:10019000BF910F9118950F931F9309B7026009BF84
:1001A00003B7016003BF09B7006809BF0FB51EB5EB
:1001B0001F7E1860026001601B7F1D7F11600FBDF4
:1001C0001EBD78941F910F910895FD0000FD0A0057
:1001D000FD1E00FD3200FD5000FD6E00FDA000FD83
:1001E000D200FDFD0000FD0000FD3200FD6400FDB9
:1001F0009600FDB400FDD200FDFD0000FDFD0032C3
:10020000FD005AFD0082FD00B9FD00FDFDFDFDFD74
:10021000B4D2FD82A0FD506E64FDFD0AD2FD32A075
:10022000FD8250FD4646FD0000000F931F93FF9393
:10023000EF93F1E0EAEC10E000916A00E00FF11FAB
:10024000E00FF11FE00FF11F059100936000059191
:1002500000936100049100936200EF91FF911F9160
:100260000F910895B7D0B0999AC0BF93AF931F93E1
:100270000F93B0E0A4E1AED0B09924C01197D9F7A4
:10028000009169000395043008F00027003041F424
:10029000B19B5F7BB1995064869B5F7D869950626C
:1002A000013011F450645F7D023011F45F7B5062C5
:1002B000033011F450645F7D009369008BD0B09BD4
:1002C000FDCF69C000916900003081F400916A009F
:1002D0000395003208F0002700936A00A6DF009320
:1002E0006E0002E000936D0097D055C0013011F50B
:1002F000B0916400A0916500D296D29613E00AEE08
:10030000A017B10710F0B0E0A1E0F894B9BDA8BD06
:100310007894B0936400A093650003E000936D00AF
:10032000B0936E0079D004E000936D00A0936E004E
:1003300073D031C0023011F5B0916600A091670012
:10034000D296D29613E00AEEA017B10710F0B0E0F3
:10035000A1E0F894BBBDAABD7894B0936600A093C9
:10036000670005E000936D00B0936E0055D006E085
:1003700000936D00A0936E004FD00DC0033059F470
:10038000052F07FF506807FD5F7701E000936D00C0
:1003900050936E0041D00F911F91AF91BF9108957E
:1003A000BF93AF93B3E0A8EE000000000000000090
:1003B0001197D1F70000AF91BF910895DF93CF93CC
:1003C000D0916B00C0916C00EBDF2197E9F7CF91E2
:1003D000DF9108950F931F932F9310916C0020913C
:1003E0006B0000E000936B0009E100936C00E6DF16
:1003F00010936C0020936B002F911F910F91089523
:100400000F93E199FECF00916D000EBBE09A0DB302
:1004100000936E000F9108950F931F931FB7E199FA
:10042000FECFF89400916D000EBB00916E000DBBE5
:10043000E198E29AE19A17FD78941F910F9108953F
:10044000D0E0CFEDCDBF2196B0E0A0E600E00D9367
:10045000AC17BD07E0F30CE107BB01EE08BB08E3F6
:1004600001BB07E802BB01E000936D00C9DF5091BA
:100470006E0002E000936D00C3DF00916E000093F8
:100480006A00D3DE03E000936D00BADF00916E00D6
:100490000093640004E000936D00B2DF00916E00F1
:1004A0000093650005E000936D00AADF00916E00E7
:1004B0000093660006E000936D00A2DF00916E00DD
:1004C00000936700002709BD08BD5F7B0BBD0ABD17
:1004D0005F7D00E000936300009369005CDEB09BE9
:1004E000C1DE00916900003091F4B19B04C072DF5D
:1004F000B199506403C06EDFB19B5F7B869B04C0E3
:1005000069DF8699506203C065DF869B5F7D03309B
:1005100009F0E5CF56FD03C050645F7D02C05F7BEC
:10052000506200E000936B000AE000936C0002E36D
:0E05300045DFB09B97DE0A95D9F7D1CF18951D
:00000001FF
